:1000000000308A00BA2800000030A1001F08C33960
:1000100021049F000D30A000A00B0C289F149F18F6
:100020000F2883161E088312A5001E08A6000430A0
:10003000A1001F08C33921049F000D30A000A00BB0
:100040001F289F149F18222883161E088312A700BA
:100050001E08A8000C30A1001F08C33921049F000E
:100060000D30A000A00B32289F149F18352883164E
:100070001E088312A9001E08AA00DA28A101A20105
:10008000A001A3013408031D48283308031962287E
:100090001030B5000310B10DB20DA00DA30D340842
:1000A0002302031D552833082002031C5E28330851
:1000B000A002031CA3033408A3020314A10DA20D84
:1000C000B50B4A2800008C28B001AF01B008031D11
:1000D0007E282F08123C031C7E2805150830A0003E
:1000E000A00B7028000005110330A000A00B76289B
:1000F00000000000AF0A0319B00A66280511D830C5
:10010000A000A00B812800002D08B2002C08B1002F
:10011000B4010A30B3003E282208AD002108AC002B
:10012000B001AF0130082D02031CA628031D9C2836
:100130002C082F020318A6280130AE000000000092
:1001400000000000AF0A0319B00A922800342C30D6
:10015000840000080319B9280230A100A001A00BF7
:10016000AF28A10BAE289730A000A00BB528800BBC
:10017000AC28002984011F3083051F1383161F1428
:100180009F141F159F15073083129F007030831630
:100190008F001B30650083121F1383161F149F14DA
:1001A0001F119F151F129F161F1383129F171F14D5
:1001B00085120428051185122808AD002708AC0017
:1001C00064200230AD00AC0164202608AD00250893
:1001D000AC0064200230AD00AC0164200230AD0000
:1001E000AC0164202A08023C031CFD28031DFC28E6
:1001F0002908ED3C031CFD2885160A30AC00A72811
:04020000D928630096
:02400E00C43FAD
:00000001FF
